:020000000528D1
:10000800882C8B1383120313831203138501860133
:100018008316FF30831603138500FF308600831292
:100028008B13063083120313A000A101A2018730AD
:1000380083168316031381008312C330A600A70119
:10004800831203138100A0308B0083160313A801C9
:10005800FF30AB01AC01AF00B000AD01AE01B100A3
:10006800B200422B83160313AA000310280DAB3EDF
:100078008400831329088000840A2A088000A80ABB
:100088002808023A0319A8010310280D8313AB3E70
:1000980084000008840A000403194328801B4328AD
:1000A80000088A0084030008820083120313D20127
:1000B800D10104305102031C6228CC288312031397
:1000C800CF015108CE000310CE0DCF0D4E08FC3ED7
:1000D8000318CF0ACE000630CF074E08CE007A2884
:1000E800831203134F088A004E0882007420831677
:1000F8000313DD0083120313CE0A0319CF0A7420F9
:1001080083120313CF00831603135D0883120313AE
:10011800CE00D0010311031992289328AB2883122B
:1001280003134F084D02031C9D28031D9D284E08EC
:100138004C02031CA028A128AB28831203134E08E5
:10014800CC02031CCD034F08CD02D00A8E2883129F
:1001580003135008003A031DB228B6280130831251
:100168000313D200D2080319BA28BB28CA2883125D
:1001780003135008303ED30083134B1883174A08E3
:10018800840053088000CA0A0319CB0AD10A5D28E3
:10019800831203134C08303ED30083134B18831784
:1001A8004A08840053088000CA0A0319CB0A83133B
:1001B8004B1883174A088400800149088A004808B8
:1001C80082008313831203134B1883174A08840091
:1001D8000008003A031DF128F72883120313CA0AFE
:1001E8000319CB0AE52803110319FB28FC28222947
:1001F8000329831203134D088A004C088200FD204E
:1002080083120313CE0083134B1883174A08840004
:100218004E08800083134B1883174A08840000088F
:10022800003A031918291929222983120313CA0A23
:100238000319CB0ACC0A0319CD0AF7288312031332
:1002480049088A00480882000430831203136A02AE
:10025800031C3229031D322900306902031835298D
:100268004629013083160313AA000030A9000000B4
:10027800A90B3B290000003083120313E902031C79
:10028800EA0328290030831203136A02031C502949
:10029800031D502904306902031853296929831260
:1002A80003136A0883160313AA0083120313690849
:1002B80083160313A9000310AA0CA90C0310AA0C97
:1002C800A90C0000A90B652900000800831203137C
:1002D80063086404031D7129812983160313AA0185
:1002E800FA30A9000000A90B76290000013083121A
:1002F8000313E302031CE4036A29080083120313AF
:10030800851508008312031385110800831203134F
:100318000515690EF03986040F38860505110800A1
:100328008621831203136308E900E90E0F30E905FB
:100338008A21831203136308E9008A2183120313B5
:10034800EA012830E90028210800822183120313DA
:100358006308E900E90E0F30E9058A2183120313C7
:100368006308E9008A2183120313EA013230E900A5
:100378002821080083160313061286120613861313
:100388008511051183120313E4010F30E3006A217C
:100398008621033083120313E9008A218312031391
:1003A800E4010530E3006A21033083120313E900F6
:1003B8008A2183120313EA016430E90028210330FB
:1003C80083120313E9008A2183120313E401053021
:1003D800E3006A21023083120313E9008A218312A1
:1003E8000313EA012830E900282128308312031377
:1003F800E3009421083083120313E30094210F30A3
:1004080083120313E3009421013083120313E300E2
:10041800942183120313E4010230E3006A210630B9
:1004280083120313E30094218312031358088A00EC
:10043800570882000C3083120313E30094218312BF
:10044800031358088A0057088200831203135A08B6
:100458000139E300E30EE30DE30DC030E30580301E
:10046800E30459083F39E30494218312031358081D
:100478008A00570882008312031359080739E300DA
:10048800E30DE30DE30DF830E3054030E304942178
:1004980083120313DC0108305C02031C542A732AFC
:1004A800831203135B08DE005A085C070318DE0A90
:1004B800DD00642A831203135E088A005D08820047
:1004C8005E2283120313E300A92183120313EA01B6
:1004D8005030E900282183120313DC0A4F2A8312C3
:1004E800031358088A005708820002308312031346
:1004F800D8008330D70001308A00BE3082008312D2
:10050800031349088A0048088200831203134A0823
:10051800D9004B08DA000230D8009730D7000230F3
:100528008A00293082008312031349088A00480888
:100538008200023083120313D800A730D70002309C
:100548008A001E3082008312031349088A00480873
:100558008200831203134A08D9004C08DB004B08B9
:10056800DA000230D800BD30D70002308A003F30B0
:10057800820083120313D901DA010230D800C9308E
:10058800D70002308A0029308200831203134908F9
:100598008A0048088200831203135908E300A9213E
:1005A8008312031358088A005708820083138312A2
:1005B80003134B1883174A0884000008003A031DE8
:1005C800E62AFD2A8313831203134B1883174A085C
:1005D80084000008D9000230D800F730D700023074
:1005E8008A00CF30820083120313CA0A0319CB0A88
:1005F800DA2A8312031349088A004808820008305F
:10060800831203134B02031C0A2B0F2B83120313B1
:100618002A08CC001E2B1030831203134B02031C34
:10062800162B1B2B831203132D08CC001E2B8312B1
:100638000313CC010730CB050130C8004B08F83E46
:10064800031C282BC801322B07390319322B03103E
:1006580083120313C80DFF3E031D2B2B4C08C8053E
:100668004808003A03090439031D0130C8003C2B2F
:10067800831203134A088A0049088200073083124C
:1006880003139F000330C9004E30C80002308A00AF
:100698007930820083120313BE01BF010730CA00FC
:1006A8000730CC003C30CB000330C9006030C800B4
:1006B80002308A00AD308200033083120313C90070
:1006C8006A30C80002308A009D3082000130840000
:1006D8008407AB3084078313B0308000840A063067
:1006E8008000831603132808013A031D7C2B432836
:1006F80083120313C30103110319832B842B822C48
:10070800831203133F08C1003E08C0000630CB0027
:100718000330CA009430C90003308A0003308200D5
:10072800831203134808C2004208003A031D9D2B98
:10073800A32B013083120313BE02031CBF0307302F
:10074800CB000330CA00AD30C90003308A00033043
:100758008200831203134808C2004208003A031DAE
:10076800B62BBB2B83120313BE0A0319BF0A3E081C
:100778004006031DC12B3F084106031DC42BFF2B58
:1007880083120313CB013430CA003F08CD003E0862
:10079800CC000330C900D530C80000308A00593079
:1007A800820083120313CB013430CA000730CD0016
:1007B8004430CC000330C900E630C80000308A005D
:1007C800E530820083120313CA01CB010330C9004C
:1007D800F230C80002308A00893082008312031385
:1007E800CB013430CA000330C900FF30C8000230E2
:1007F8008A00DA30820083120313CA010130CB0069
:100808000430C9000C30C80002308A0089308200E8
:10081800831203134308C200C20DC201C20D033084
:10082800C2050730C500383042070318C50AC4009E
:10083800232C8312031345088A00440882001D24D0
:1008480083120313D9000430D8002F30D7000230A8
:100858008A00CF308200831203134308C200C20EFD
:10086800C20CC20C0330C2050330C2050730C500F4
:10087800383042070318C50AC400482C83120313F2
:1008880045088A0044088200422483120313D900D1
:100898000430D8005430D70002308A00CF308200AC
:1008A800831203134308C200C20EC20C0730C205EC
:1008B8000330C2050730C500383042070318C50A9F
:1008C800C4006C2C8312031345088A004408820074
:1008D800662483120313D9000430D8007830D70077
:1008E80002308A00CF30820083120313C30A81309A
:1008F80083160313A900043036287F2B83120313B1
:1009080033088A0032088200FF00030E831603139F
:1009180083160313A000A00E0A08A1000408A20071
:100928000B1DB02C26088312031381005030831648
:100938000313A707B4300318013EFF3A013EA6008F
:100948000B11FF30B01BAB2CAF07031CB007B21B59
:10095800B02CB107031CB2077C08A3007D08A400D3
:100968007E08A5002508FE002408FD002308FC00D9
:100978002208840021088A0020088300FF0E7F0EC9
:100988000900831603134D08D0004C08013E0318D4
:10099800D00AD001831384000008013ECF008313DE
:1009A8004D1883174C08840000084F020318DD2CEB
:1009B800E02C83160313CF014D08D1004C08023EEA
:1009C8000318D10A831351188317840000084F06AF
:1009D8000319EF2CF62C013083160313C900C9093B
:1009E800C90A222D831603134D08D1004C08013E75
:1009F8000318D10A8313511883178400D101000802
:100A0800033E0318D10A4C07D0000318D10A4D0839
:100A1800D107831351188317500884004E088000AB
:100A28004D08D1004C08013E0318D10A8313511810
:100A3800831784004F088000C901222D83160313F1
:100A48004B088A004A08820083120313AA01AB01EB
:100A580083160313350883120313AC00AD01AE01EE
:100A680083160313360883120313AF008316031388
:100A78003508850436088604043083120313A90058
:100A880083160313380883120313B1008316031364
:100A9800370883120313B0008316031334088A003F
:100AA800330882008312031330083104031D5D2DBF
:100AB800992D013083160313C200C3010830430285
:100AC800031C672D992D831603133F084205003A2E
:100AD800031D6F2D932D8316031343084107C4008C
:100AE80040084205003A031D7A2D7D2D8316031315
:100AF800C41783120313310883160313CD0083121E
:100B08000313300883160313CC004408CE000530C5
:100B1800CB009330CA0004308A00C530820003102D
:100B280083160313C20DC30A622D831603133E08EE
:100B38008A003D088200831203132C08003A031D23
:100B4800A62DF92D83120313050883160313B80085
:100B580083120313050883160313B70083120313C4
:100B6800050883160313B8048312031305088316B4
:100B78000313B70583120313050883160313B80478
:100B880083120313050883160313B705831203138F
:100B98002B0883160313B600831203130508AB0052
:100BA800831603133608831203132B0683160313C5
:100BB800B500831203132B0883160313B80483129A
:100BC80003132B0883160313B70538083706B60036
:100BD80036083504831203132C05003A031DF52D3E
:100BE800F92D033083120313A9002F08003A031DBF
:100BF800FE2D512E83120313060883160313B80023
:100C080083120313060883160313B7008312031312
:100C1800060883160313B804831203130608831601
:100C28000313B70583120313060883160313B804C6
:100C380083120313060883160313B70583120313DD
:100C48002E0883160313B600831203130608AE009A
:100C5800831603133608831203132E068316031311
:100C6800B500831203132E0883160313B8048312E6
:100C780003132E0883160313B70538083706B60082
:100C880036083504831203132F05003A031D4D2E31
:100C9800512E033083120313A9002908003A031DBB
:100CA800562EAA2EFF3083120313A9072908003AEB
:100CB80003195F2EAA2E831203132A082B062C056C
:100CC80083160313B5003508003A031D6C2E842ED5
:100CD800831203132B082C05AA0083160313350867
:100CE800BF00831203132A0883160313C000C1012F
:100CF8000630BE008430BD0005308A0056308200C0
:100D0800831203132D082E062F0583160313B5002F
:100D18003508003A031D912EAA2E831203132E08BC
:100D28002F05AD00831603133508BF008312031384
:100D38002D0883160313C0000830C1000630BE001A
:100D4800AA30BD0005308A0056308200831603138E
:100D580034088A0033088200C03083160313B500B4
:100D6800B601B8012030B7000630B400C030B30077
:100D780005308A002830820003110319C42EC52EBD
:100D8800F22E063083160313B400CF30B3000530BB
:100D98008A009F30820083160313A901AA0128083C
:100DA80084008407AF3084078313840A8017840380
:100DB80029088000840A2A088000E630A900063045
:100DC8003628432883160313280884008407AF3085
:100DD80084078313840A801FE52EC02E70088A00BA
:100DE800831203136F088200643400340A34003419
:100DF80010342734E8340334643400340A340034BB
:100E08000034CA349A343B340034E134F5340534C0
:100E18008034963498340034403442340F340034EB
:100E2800A0348634013400341034273400340034BC
:100E3800E8340334003400346434003400340034BB
:100E48000A3400340034003430343134323433342A
:100E58003434353436343734383439344134423420
:100E680043344434453446347C342F342D340734E9
:100E780010340834083404340234023401340034A1
:0A0E880020342034203420340034DC
:02400E00103F61
:00000001FF
